:02000000902846
:020008000800EE
:1000100052206F206720652072202020422065201A
:1000200065207020202031202E2030202C20202000
:100030004F20452039204D204B2056202C202020B9
:100040002820632029202020322030203020322018
:100060009000193091006400910B3328900B3128D7
:1000700000341408920015089300851403303020D2
:10008000851003303020930B3D28920B3B28003421
:100090000230940096309500051539200511003482
:1000A00001309400643095000515392005110034A5
:1000B0000511FF303020FF30302064303020003414
:1000C00002309400963095003920003448205820A2
:1000D00050205820482058200034502058205020CC
:1000E0005820482058204820582050205820502080
:1000F00058200034502058204820582050205820A4
:100100000034502058205020582050205820502093
:100110005820582058205020582050205820003473
:1001200083168113FF30860000308500011383128F
:1001300085018B010B168B15630000000B18BA2884
:100140008B18A32897288B100514FF303020FF3020
:1001500030206400061CA928861C6020061D66202D
:10016000861D6D20061E7A20861E812005108510B2
:10017000051197280B10FF303020061FC528861F59
:10018000CC28051085100511972805146400061B5E
:10019000BA2850205820C62805146400861BBA28A7
:0601A00048205820CD2884
:02400E00F93F78
:00000001FF
